:020000040000FA
:020000000528D1
:0800080005288B010730990067
:100010008316FF308500851205128101043095009A
:10002000FF2390008312850105168512DB209E2098
:100030000330A300AF20FF30A300AF20CC209E20D0
:10004000BB30A300AF20A301AF20CC209E201030F6
:10005000A300AF200830A1008030A300AF20A10B87
:100060002C28CC209E20B730A300AF20D230A30094
:10007000AF20CC209E200F30A300AF20A301AF20E3
:100080004F30A300AF20CC209E201830A300AF201B
:10009000A301AF20A301AF200430051D0230A3004F
:1000A000AF20E230051D7130A300AF20A301AF20C7
:1000B0000C30051D0B30A300AF202330051DB730D9
:1000C000A300AF20A301AF20A301AF209A30051DEC
:1000D0003930A300AF200930A100A301AF20A10B4C
:1000E0006D280130A300AF20A301AF201F30051DF4
:1000F0001E30A300AF202F30A100A301AF20A10B21
:100100007D28CC209E209530A300AF201630A10082
:10011000A301AF20A10B8828CC209E20B130A300E2
:10012000AF20AC30A300AF20CC209E200330A30032
:10013000AF20FE30A300AF20CC206300A320C0304E
:10014000A300AF200800831605128312051685163A
:100150000000051200008512000005160800831635
:10016000051283120830A2000310A30D031CBA2845
:100170000516BB2805128516000000008512A20B8B
:10018000B5280516C42008008316051683128516A7
:10019000000000008512080000008316051283127B
:1001A0000512000000008516000000000516000082
:1001B0000000851208001430A000E0280230A000E2
:0E01C000A430A100A10BE228A00BE02808004B
:02400E00C43FAD
:00000001FF
